:020000040800F2
:1000000000040120010200082D0D00082D0D00083C
:100010002D0D00082D0D00082D0D00082D0D0008D8
:100020002D0D00082D0D00082D0D0008E92B0008EE
:100030002D0D00082D0D00082D0D00082D0D0008B8
:100040002D0D00082D0D00082D0D00082D0D0008A8
:100050002D0D00082D0D00082D0D00082D0D000898
:100060002D0D00082D0D00082D0D00082D0D000888
:100070002D0D00082D0D00082D0D00082D0D000878
:100080002D0D00082D0D00082D0D00082D0D000868
:100090002D0D00082D0D00082D0D00082D0D000858
:1000A0002D0D00082D0D00082D0D00082D0D000848
:1000B000D52400082D0D00082D0D00082D0D000879
:1000C0002D0D00082D0D00082D0D00082D0D000828
:1000D0002D0D00082D0D00082D0D00082D0D000818
:1000E0002D0D00082D0D00082D0D00082D0D000808
:1000F0002D0D00082D0D00082D0D00082D0D0008F8
:100100002D0D00082D0D00082D0D00082D0D0008E7
:100110002D0D00082D0D00082D0D00082D0D0008D7
:100120002D0D00082D0D00082D0D00082D0D0008C7
:100130002D0D00082D0D00082D0D00082D0D0008B7
:100140002D0D00082D0D00082D0D0008512200086E
:100150002D0D00082D0D00082D0D00082D0D000897
:100160002D0D00082D0D00082D0D00082D0D000887
:100170002D0D00082D0D00082D0D00082D0D000877
:100180002D0D00082D0D00082D0D00082D0D000867
:100190002D0D00082D0D00082D0D00082D0D000857
:1001A0002D0D00082D0D00082D0D00082D0D000847
:1001B0002D0D00082D0D00082D0D00082D0D000837
:1001C0002D0D00082D0D00082D0D00082D0D000827
:1001D0002D0D00082D0D00082D0D00082D0D000817
:1001E0002D0D00082D0D00082D0D00082D0D000807
:1001F0002D0D00082D0D00082D0D00082D0D0008F7
:1002000072B6374880F3098836484EF60851CEF268
:100210000001086040F20000CCF200004EF634719C
:10022000CEF200010860BFF34F8FBFF36F8F40F233
:100230000000C0F2F0004EF68851CEF200010860D6
:10024000BFF34F8FBFF36F8F4FF00000E1EE100A46
:100250004EF63C71CEF200010860062080F314884F
:10026000BFF36F8F00F008FD02F076F94FF05530C4
:100270001D491E4A91423CBF41F8040BFAE71C4954
:10028000174A91423CBF41F8040BFAE719491A4A50
:100290001A4B9A423EBF51F8040B42F8040BF8E7A0
:1002A00000201749174A91423CBF41F8040BFAE776
:1002B00000F022FD02F052F9134C144DAC4203DA67
:1002C00054F8041B8847F9E700F03EF8104C114D34
:1002D000AC4203DA54F8041B8847F9E700F00ABD82
:1002E0000008012000000008000001200004012097
:1002F00000040120A8360008000801205008012051
:1003000050080120601A01200002000800020008C5
:1003100000020008000200082DE9F04F2DED108AC0
:10032000C1F80CD0D0F80CD0BDEC108ABDE8F08F2D
:10033000002383F311882846A047002000F000FF27
:1003400000F096FE00DFFEE738B5184B79221A70F0
:100350006FF07F0200245A720E225C709C70DC7079
:100360001C715C719C71DC711C729A72DC7202F0FF
:1003700055FB0F4B984217D00133984241F2883415
:1003800012BF002500240125002002F04DFB0DB115
:1003900000F052F800F044FC00F034FB204600F07E
:1003A000B9F800F049F8F9E72546EDE750080120D3
:1003B000010007B008B500F0C7FAA0F120035842C9
:1003C000584108BD07B5054B02211B88ADF8043024
:1003D00001A800F007FB03B05DF804FB7C330008C4
:1003E00010B51148C3680BB100F06CFD0F4C104AFA
:1003F0000D4800234FF47A7100F028FD236813B1F3
:100400002368013B2360636813B16368013B636049
:10041000084B1B7833B9636823B9022000F0BAFB9C
:100420003223636010BD00BF5C080120740D012001
:10043000E1030008700801202DE9F0412F4C2368EA
:10044000013359D02E4D2F4B2A689A4254D92E4B46
:100450009B6803F1006303F5C0339A424CD200203D
:1004600000F0ECFA294B0220187000F08BFB72B6FA
:10047000274B1C6026682D68BFF34F8FBFF36F8F2B
:10048000083B0022C3F88420BFF34F8FD3F88020AD
:100490005969C2F3C90421F48031C2F34E32596163
:1004A0005201A70743F6E07E02EA0E0838462146CD
:1004B000013948EA000CB1F1FF3FC3F874C200F102
:1004C0004040F5D1203A12F1200FEDD1BFF34F8F0C
:1004D000BFF36F8FBFF34F8FBFF36F8F5A6922F453
:1004E00000325A610022C3F85022BFF34F8FBFF38E
:1004F0006F8F86F308882847BDE8F08100800108E7
:1005000004800108FF7F01085008012070080120C5
:1005100008ED00E02DE9F04FBD4B0546BD489C6855
:1005200000228FB0C26072B6202282F3118862B6B8
:10053000C26898460AB100F0C5FC0023B64AB54827
:100540004FF47A7100F082FC002383F31188DFF806
:10055000E4920DB1C9F80050B04EC9F804303370C0
:100560004FF0FF37012000F00DFB002D00F0AF81B0
:10057000D9F80030002B40F0AA810FB0BDE8F08F11
:100580000220FFF717FF00283AD1A54B1B88ADF8D2
:100590002430022109A800F025FAE3E74FF47A702D
:1005A00000F0D2F9B0F1000BEFDB0220FFF702FF01
:1005B0000028EAD00BF1FF300428E6D8DFE800F08D
:1005C00003090E1114000EA8052340F8143D042160
:1005D00001E08F48042100F005FA11E00421914860
:1005E000F9E704219048F6E71C25284600F028FA90
:1005F00004350990042109A800F0F4F92C2DF4D158
:1006000000F004FBFFF7DEFE5FE10220FFF7D2FE01
:100610000028BAD0012000F011FA0220307000F05A
:10062000B1FA4FF0000B5FFA8BFA504600F01EFA59
:100630000BF1010B044618B1504600F027FAF2E71F
:1006400001230220337000F093FAD8F808309C425E
:1006500007D2204600F0F4F9013040F0198104344B
:10066000F3E700243470C9F80440C9E70220307071
:1006700000F088FA322000F067F9B0F1000B84DB5B
:100680001BF0030381D1D8F808100BEB04028A4257
:100690003FF67BAFBBF5807F3FF677AF634A9A4664
:1006A000DA4501920FDA4FF47A7000F04DF90390B9
:1006B00003990029FFF669AF019A03990AF802101D
:1006C0000AF1010AECE7C820FFF774FE00283FF4A6
:1006D0005CAF24B9554B4FF0FF321F681A60534B83
:1006E0002BF0030BA344A3EB040A5C4588D05AF813
:1006F0000410204600F0AAF9204600F0A1F95AF8AB
:100700000420904240F0C4800434EEE70220FFF75A
:1007100051FE00283FF439AF4FF0000B5D46D8F88A
:1007200008309B4534D2BBF1000F14D17A1C12D093
:1007300009973F494B689BB1002209A8135C6B40A5
:10074000DBB2013251F82330042A83EA1525F5D1B2
:100750000BF1040BE3E7584600F072F90990E8E763
:100760001A46082012F0010F4FEA52021FBF82F012
:100770006D4282F4380282F4034282F02002013892
:10078000F0D141F823200133B3F5807FE8D1D3E7DE
:100790000EA840F8285D1AE70EA8002340F8143D83
:1007A000642100F0FBF800287FF4EFAE0220FFF791
:1007B00001FE00283FF4E9AE099800F079F90EAB8C
:1007C00043F8240D0421184605E70EA8002340F83D
:1007D000143D642100F0E2F800287FF4D6AE022038
:1007E000FFF7E8FD00283FF4D0AE099800F06EF95D
:1007F0000EAB43F8200DE5E70220FFF7DBFD0028F4
:100800003FF4C3AE00F068F90EAB43F81C0DD9E716
:10081000500801205C080120E10300087008012055
:100820007E33000854080120580801207408012074
:1008300074090120740D01200220FFF7BBFD002880
:100840003FF4A3AE09A9142000F04CF905460EA808
:10085000042140F8185D00F0C5F8294609A8BAE659
:100860004FF47A70FFF7A6FD00283FF48EAE7B1C94
:1008700005D1FFF7A7FD324800F06AFC7DE6394656
:10088000002000F0E3F8002000F0DAF88742F0D012
:100890002C4B7BE60EA8002340F8143D642100F0A9
:1008A0007DF800287FF471AE0220FFF783FD002859
:1008B0003FF46BAEFFF786FD41F2883000F048FC54
:1008C000099800F0D7F900F0A1F900254AE60020C8
:1008D00000F03AF80390039B002BFFF646AE012090
:1008E00000F046F9039B213B122B3FF63BAE01A2E1
:1008F00052F823F0810500089D0500080B0600084A
:100900006505000865050008650500086D06000816
:10091000650500080D07000899070008CB070008C7
:10092000F907000865050008390800086505000892
:100930006108000801060008650500089508000820
:10094000A08601008033000837B5114A12780132C1
:10095000D2B20024012A03468DF8074011D80D4871
:100960000268D5694FF47A7253430DF107010122F1
:10097000A847012805D1084B9DF807001C7003B05B
:1009800030BD4FF4FA7000F0E3FB4FF0FF30F6E7B4
:100990000008012018110120800D012038B50E4BF0
:1009A0001A780132D2B2012A05460ED80B480368E4
:1009B000DC694FF47A734B4304222946A04704288C
:1009C00003D1074B0020187038BD4FF4FA7000F0C7
:1009D000BFFB4FF0FF3038BD000801201811012087
:1009E000800D012030B4054C23689D69044B0A46F4
:1009F000AC460146204630BC604700BF18110120BC
:100A0000A0860100F8B501F02DFF094C094E0A4FF0
:100A10002070002530682378834207D901F01CFF3D
:100A2000336805440133BD423360F3D9F8BD00BFDC
:100A3000810D01207C0D0120FF7F010001F0DABF54
:100A400000F1006000F5C0300068704707B502ABE8
:100A500000F1006043F8041D0422194600F5C0307F
:100A600001F056FF03B05DF804FB0000054B1A6867
:100A7000054B1B781344834202D9104401F0ECBEAD
:100A8000002070477C0D0120810D012038B5074DF5
:100A900004462868204401F0E7FE28B9286820446D
:100AA000BDE8384001F0F8BE38BD00BF7C0D012024
:100AB00010F0030308D1B0F5806F05D800F10050A5
:100AC000A0F571200068704700207047014BC058A6
:100AD000704700BF20F4F01F014B1868704700BF3B
:100AE000002004E0F0B5204B1E68204B1F885D6895
:100AF00093F90840C6F30B02BA424FEA164622D0D9
:100B00009F89BA4221D01F8BBA4206D102220C24FF
:100B100004FB02335D6893F90840B6F5805F16D098
:100B200041F201039E4208BF5A24421E0A44013D7D
:100B30000B46934215D215F9016F581C4EB103466E
:100B400000F8016CF5E70022E1E70122DFE741242C
:100B5000EBE72C2582421D7001D9981C5C70401A6D
:100B6000F0BD1846FBE700BF002004E004080120A8
:100B7000022802BF024B4FF480229A61704700BFE7
:100B800000000240022802BF014B04229A61704714
:100B900000000240022801BF024A536983F00403A7
:100BA000536170470000024010B50023934203D008
:100BB000CC5CC4540133F9E710BD000030B5441ECD
:100BC00014F9010F0B4660B193F90050854201F111
:100BD000010106D11AB993F90020801A30BD013AFB
:100BE000EEE7002AF7D1104630BD0000024603466A
:100BF000981A13F9011B0029FAD1704702440346E1
:100C0000934202D003F8011BFAE77047024B1A78AF
:100C1000024B1A70704700BF800D012000080120B0
:100C200038B5104D104C284600F05AFB2146284696
:100C300000F082FB23680D48DA6ED2F8043843F0E6
:100C40000203C2F8043800F083FA0949206800F072
:100C500093FC2368DA6ED2F8043823F00203C2F85A
:100C6000043838BD181101209435000840420F00A7
:100C7000E435000870470000F0B5BFF34F8FBFF3B5
:100C80006F8F1B4B0021C3F850125A6942F4003297
:100C90005A61BFF34F8FBFF36F8FC3F88410BFF358
:100CA0004F8FD3F88020C2F3C904C2F34E325201F1
:100CB000A50743F6E07602EA060E284621464EEAEC
:100CC00000070139C3F860724F1C00F14040F6D1B3
:100CD000203A12F1200FEED1BFF34F8F5A6942F440
:100CE00080325A61BFF34F8FBFF36F8FF0BD00BFEB
:100CF00000ED00E0FEE70000084A094B09498B427D
:100D000004D3094A0021934205D3704752F8040FD7
:100D100043F8040BF3E743F8041BF4E7F436000848
:100D2000601A0120601A0120601A01201EF0040FD1
:100D30000CBFEFF30880EFF309808169004A104788
:100D4000490D000870470000204B02681A60204BD4
:100D500042681A601F4B82681A601F4BC2681A6093
:100D60001E4B02691A601E4B42691A601D4B826954
:100D70001A601D4BC2691A601C4B1D491A681D4B35
:100D80001A601A68120A0A701A681B4B1A701B4BF9
:100D90001A681B4B1A601B4B1A681B4B1A601B4BC3
:100DA0001A681B4B1A601B4B1A681B4B1A601B4BB3
:100DB0001A681B4B1A601B4B5A6A1B4B1A601B4B61
:100DC0001B68DB0701D500BEFEE7FEE7B40D01207E
:100DD000B80D0120C00D0120C40D0120BC0D012063
:100DE000A80D0120AC0D0120B00D012028ED00E080
:100DF0008C0D0120900D0120A00D01202CED00E0B4
:100E0000980D012030ED00E0940D01203CED00E054
:100E1000840D012034ED00E09C0D012038ED00E050
:100E2000880D012000ED00E0A40D0120F0ED00E0B0
:100E3000054B03F114025A619A614FF0FF32DA61F7
:100E400000221A62704700BFC80D0120F8B5036187
:100E50004FF08043C2605C6A194B1A46022952F86F
:100E6000145F38BF0221954206461F460AD15861D9
:100E700098611C620560456081600819BDE8F84012
:100E800000F050BB186AAB68241A0C1902D3E41A9C
:100E90002D6804E09C4202D2204400F051FBAB6874
:100EA0009C42F4D86B68736035601E606E60B460FD
:100EB000A9684FF0FF33091BA960FB61F8BD00BFB3
:100EC000C80D012010B41B4C234653F8141F814257
:100ED00010D0416802680A60026851609A424FF07F
:100EE0000001C16003D0936881680B4493605DF892
:100EF000044B70470A68626100209A425360C860E0
:100F000003D15DF8044B00F015BB93688868034477
:100F100093604FF08042506A226A821A9342E6D967
:100F20009B1A022B2CBFC01802305DF8044B00F056
:100F300007BB00BFC80D0120024B00221B605B6095
:100F40009A607047C80D0120002303748268054B26
:100F50001B6899689142FBD25A6803604260106036
:100F600058607047C80D012008B572B6202383F37E
:100F7000118862B6037C032B05D0042B0DD02BB94E
:100F800083F3118808BD436900221A604FF0FF33D4
:100F90004361FFF7D9FF0023F2E790E80C001A60E5
:100FA00002685360F2E70000002303748268054B77
:100FB0001B6899689142FBD85A68036042601060D0
:100FC00058607047C80D0120054B196908741868EE
:100FD00002681A605360186101230374FFF79CB91B
:100FE000C80D012030B54B1C87B005460A4C10D007
:100FF00023690A4A01A8FFF729FF2846FFF7E4FF03
:10100000049B13B101A8FFF75DFF2369586907B07E
:1010100030BDFFF7D9FFF8E7C80D0120690F0008C0
:1010200038B50C4D41612B6981689A68914204463C
:1010300003D8BDE83840FFF787BF1846FFF784FFA5
:1010400001232C61014623742046BDE83840FFF798
:1010500063B900BFC80D0120044B1A681B69906872
:101060009B68984294BF002001207047C80D012062
:1010700010B5084C236820691A6822605460012268
:1010800023611A74FFF790FF01462069BDE8104004
:10109000FFF742B9C80D012008B5FFF7DDFF18B111
:1010A000BDE80840FFF7E4BF08BD000072B620238A
:1010B00083F3118862B670478260022202740022B4
:1010C00042748261704700008368A3F1840243F890
:1010D000142C026943F8442C426943F8402C084A16
:1010E00043F8242CC26843F8182C022203F8102C71
:1010F000002203F80F2C43F8082CA3F120007047BE
:101100003103000808B5FFF7DFFFBDE80840FFF72F
:101110001BBF000010B5FFF7C9FFFFF7D5FF002187
:101120000446FFF77DFF002383F31188204610BD9E
:10113000024B1B6958610F20FFF746BFC80D012005
:1011400008B5FFF7B3FFBDE80840FFF7F1BF0000A7
:1011500008B50146FFF7AAFF0820FFF743FF002369
:1011600083F3118808BD000010B5054C23690360A6
:1011700058610320FFF728FF2369586910BD00BF9D
:10118000C80D012003682BB1002202605961184686
:10119000FFF7DABE7047000049B1064B42681B6991
:1011A00018605A60136043600420FFF71BBF4FF0C4
:1011B000FF307047C80D01200368984206D01A68B6
:1011C0000260506059611846FFF7BEBE70470000CC
:1011D00038B504460D462068844200D138BD036806
:1011E00023605C604561FFF7AFFEF4E772B6202331
:1011F00083F3118862B6704713B5446BD4F88C340E
:101200001A681178042916D1217A022913D1197983
:10121000128901238B4013420DD101A904F144002E
:1012200001F042FE024630B1D4F88C44019B217992
:10123000206800F0F1F902B010BD00000C3001F0A0
:10124000B3BD00004FF0FF330C3001F0ADBD000026
:10125000443001F095BE00004FF0FF33443001F000
:101260008FBE00000C3001F083BD00004FF0FF3155
:101270000C3001F07DBD0000443001F061BE000083
:101280004FF0FF32443001F05BBE0000D0F88C24F8
:1012900038B5136819780429054601D0012038BDF6
:1012A000017A0229FAD112795C8901209040044028
:1012B000F4D105F10C0001F015FD02460028EDD037
:1012C000D5F88C544FF480732868697900F092F94E
:1012D000204638BD406BFFF7D9BF000070470000C3
:1012E0007FB50346114A43F8042B012543600226CB
:1012F0000F4B057204460290019300F17C022946CF
:1013000000964FF480730C3001F0C8FC094B019338
:10131000029400964FF4807304F52172294604F17B
:10132000440001F09DFD04B070BD00BFB033000863
:10133000D5120008F911000808B50A68FFF756FF32
:101340000B7902EB830318624B790D3342F82300CB
:101350008B7913B102EB8302106202230372C0F88F
:101360008C14002383F3118808BD000038B50446AF
:1013700001250221043001F013FC04F10C00257555
:101380006FF00101FFF724FF84F84C5004F1440092
:101390006FF00101BDE83840FFF71ABF10B5012119
:1013A0000446043001F0FCFB0023237584F84C3024
:1013B00010BD000038B5044600250C3001F086FC55
:1013C00004F14400257501F063FD201D84F84C50A4
:1013D000012101F0E5FB2046BDE83840FFF756BF8C
:1013E00090F85C3003F06003202B19D190F85D2059
:1013F000212A0AD0222A4FF000030ED0202A0FD132
:10140000084A02650722426504E0064B036507238C
:101410004365002383650120704703654365F9E751
:101420000020704728080120D0F88C3437B51A689E
:101430001178042904461AD1017A022917D11979A1
:10144000128901238B40134211D100F14405284633
:1014500001F0F2FD58B101A9284601F025FDD4F8AC
:101460008C44019B21790246206800F0D5F803B036
:1014700030BD000000EB8103F7B51C6A05460E463F
:10148000ECB105EB8607FFF7B1FE201D082101F046
:1014900087FBFB685B691B68443413B1204601F08D
:1014A00011FD01A9204601F0FFFC024648B1019B55
:1014B0003146284600F0B0F8002383F3118803B0CA
:1014C000F0BDFB685A691268002AF5D01B8A013BFF
:1014D0001340F1D105F15C02EAE700000D3110B5CF
:1014E00050F82140C4B1FFF781FE0421601801F0DB
:1014F00057FBD4F88C241368527903EB820304F170
:101500000C00DB689B69596801F0F6FB2046FFF789
:10151000BDFE002383F3118810BD0000704700005A
:1015200000F0EEBF4FF08043002258631A610222A0
:10153000DA6070474FF080430022DA6070470000A5
:101540004FF080435863704772B6202383F31188AD
:1015500062B6704700F0A2BB012303700023436012
:1015600000F1240200F1380142F8043B8A42136181
:10157000FAD103814381704738B50446FFF7E4FF91
:1015800000254160C560056145618561C5610562F1
:1015900000F098FB0223237085F3118838BD00000A
:1015A00070B500EB810305465069DA600E461446BB
:1015B00018B110220021FFF721FBA06918B11022F9
:1015C0000021FFF71BFB31462846BDE8704000F0C4
:1015D00053BC0000028902F001020281428902F03C
:1015E000010242810022026142618261C2610262A3
:1015F00000F0D6BCF0B400EB81044789E468012513
:10160000A4698D403D43458123600023A26063604F
:10161000F0BC00F0F1BC0000F0B400EB81040789DD
:10162000E468012564698D403D4305812360002302
:10163000A2606360F0BC00F06FBD000070B50223D3
:10164000002504460370A0F8645080F8665080F8C6
:10165000675005814581C560056145618561C5614A
:10166000056280F84C5000F0A5FB63681B6823B14D
:1016700029462046BDE87040184770BD436802788F
:101680001B6880F86820052202700BB104211847FE
:1016900070470000436890F868201B6802700BB127
:1016A000052118477047000070B50023044680F8F4
:1016B0004C3000F15C0200F095FC63689B685BBBFA
:1016C00094F85C5015F0600614D194F85D3005F084
:1016D0007F0545EA0325B5F5407F00F0A38057D884
:1016E000022D00F0EE803DD8002D00F08580012D08
:1016F00000F0E1800021204600F0CEFE00212046CF
:1017000000F0C0FE63681B6813B1062120469847AD
:10171000062384F84C3070BD204698470028CFD06F
:1017200094F8632094F8623043EA0223626D934296
:1017300038BF636594F95C30656D002B80F20081E1
:10174000002D00F0EF80012384F84C30FFF7FCFE01
:10175000636D226D00212046FFF75EFF002383F3B7
:10176000118870BDB5F5807F4DD0B5F5817FC1D1B1
:1017700094F85E30002BBDD194F8603013F00F0167
:1017800026D01A06204640F1B68000F099FE1FE0F0
:10179000B5F5C06F50D020D840F202339D4200F022
:1017A000AD80B5F5A06FA5D1B4F85C30B3F5A06FEE
:1017B0000ED194F85E3084F86630204600F050FB7D
:1017C00063681B6813B101212046984703232370E7
:1017D000002323656365A365A2E7B5F5106F41D0CB
:1017E00040F602439D4266D0B5F5006F82D104F108
:1017F00067032365012333E004F1640323650223B7
:101800006365A5658CE794F85E30012B7FF472AFB9
:10181000B4F8643023F00203A4F8643026656665EA
:10182000A6657DE794F85E30012B7FF463AFB4F8D2
:10183000643043F00203EFE794F86120616894F8A4
:1018400060304D6894F85F1043EA0223204694F814
:101850005E20A84700283FF44DAF43682365036826
:101860006365DDE794F8672094F85E309A42AFD064
:101870002378042B0FD1FFF767FE2046FFF7AAFE5F
:1018800086F31188636884F867601B680321217000
:101890000BB12046984794F85E30002B98D084F81E
:1018A00067300423237063681B68002B90D00221EB
:1018B000204698478CE72F4B23650223636500235E
:1018C00089E794F8601011F0800F204601F00F01B5
:1018D0000ED000F079FB012806D002287FF40AAF71
:1018E000254B236560659BE7244B2365656597E77A
:1018F00000F05CFBEFE700F0D9FD69E794F85E309B
:10190000002B7FF4F7AE94F8603013F00F013FF432
:101910005FAF1B06204602D500F0BEFD58E700F081
:10192000B1FD55E7032384F84C30FFF70DFE2B463D
:101930002A4629462046FFF75DFE85F3118870BDD3
:101940005DB1042384F84C30FFF7FEFD636D226D1A
:1019500000212046FFF74EFE00E7052384F84C30B7
:10196000FFF7F2FD2B462A4629462046FFF754FE94
:10197000E3E700BFD8330008D0330008D4330008B1
:1019800038B590F84C300446062B21D8DFE803F038
:10199000350421353530350090F8631090F8622019
:1019A000436D42EA01229A4213D9C268128AB3FBFC
:1019B000F2F502FB153565B9FFF7C6FD2B462A4641
:1019C0002946FFF729FE85F31188022384F84C305D
:1019D00038BD032384F84C30FFF7B6FD00231A46C8
:1019E00019462046FFF706FE002383F3118838BD11
:1019F000836D03B198470023E8E7002100F04CFD18
:101A00000021204600F03EFD63681B6813B10621EB
:101A1000204698470623D9E790F84C20062A38B587
:101A2000044620D80123934013F0670F1CD113F014
:101A300008050ED1DB0616D5052380F84C30FFF7DC
:101A400083FD2B462A462946FFF7E6FD85F31188DC
:101A500038BDC3689B695B682BB9836D03B1984738
:101A6000002384F84C3038BD002100F015FD002122
:101A7000204600F007FD63681B6813B1062120466D
:101A800098470623EDE7000072B6202383F3118800
:101A900062B67047036F30B500229D68C46E114670
:101AA0004FF0FF3004EB421301329542C3F80019A6
:101AB000C3F81019C3F80809C3F8001BC3F8101BBA
:101AC000C3F8080BEED24FF00113C4F81C3830BD38
:101AD000890141F02001016103699B06FCD41220B9
:101AE00001F040B82DE9F04F87B00446C56EFFF70E
:101AF000CBFF00F17C0305934FF0000B2378012B03
:101B000004D0A36F4BB96B69DB0606D4AB690598AB
:101B100043F01003AB61FFF727FB8BF311884FF005
:101B20000008236F9B685FFA88F083421AD2FFF7A0
:101B3000ABFFE3E7E66E336A03F4F012B2F5802FF1
:101B400066D0B2F5402F0DD1C3F30A1103F00F0395
:101B500004EB830306F58056DB681F6A00231A46F0
:101B6000994248D1696911F01001E3D1012303FAC8
:101B700000F2A36F1A4200F08C80FFF785FFAB687C
:101B800023F00103AB60A36F23EA0203A36781F391
:101B9000118804EB8003D3F80CC0431CDCF814104C
:101BA0001B030293D1F80090430104934868484511
:101BB00060D2BCF81060E76EA9EB0003B34228BF07
:101BC0003346049EBE19D6F81869B6B2B3EB860F39
:101BD00062D8029EBE1903968E680196A6F1040A89
:101BE0009E46039E5AF8047F3760BEF1040F3BD92E
:101BF000AEF1040EF5E713F0030F08BF3268072BB0
:101C000098BF3A7003F101039CBF120A0137A7E79E
:101C1000C3F30A1103F00F0304EB830306F58056A8
:101C2000DA6892691768D2F808C05268A7EB020E0A
:101C300000221746914208D1DB689E69B26873683A
:101C40000A440B44B26073608CE712F0030F08BFC4
:101C50003768964588BF8CF8007002F1010284BF96
:101C60003F0A0CF1010CE5E7019E1E4403448E601F
:101C70004B609BE70121FFF707FFAB6843F00103CF
:101C8000AB6021B9D5F834381A43C5F834288BF342
:101C9000118808F1010844E70021ECE710B5074C72
:101CA0002046FFF759FC4FF0A0420023E266044AA9
:101CB000E3672267C4F8803010BD00BF100E01201A
:101CC0000034000870B50378012B86B005465DD15D
:101CD000304BC46E984213D12F4B5A6B42F08002A6
:101CE0005A635A6942F080025A6100225A610E21F9
:101CF000432001F0C1F9294BE360294BC4F80038B7
:101D00000023AB67C4F8003EC02323604FF40413E4
:101D1000A363EE6E202000F025FF012333613369B9
:101D2000DB07FCD4122000F01DFF3369002BFCDA26
:101D30000026A6602846FFF7ADFE6B68C4F8106861
:101D4000DB68C4F81468C4F81C680BBB154BA361AE
:101D50004FF0FF336361D5F880309BB9124B00938D
:101D600005F18803019305F53C7302930223039365
:101D700068460E4B04930595FFF7C4F9C5F880003B
:101D8000FFF78AF9A36843F00103A36006B070BDB2
:101D9000074BDCE7100E01200038024040140040E1
:101DA00003002002003C30C00C340008E51A000893
:101DB000083C30C0F8B5C46E054600212046FFF748
:101DC00087FE296F00234FF001128F68C4F8343862
:101DD0004FF00066C4F81C284FF0FF3004EB4312AC
:101DE00001339F42C2F80069C2F8006BC2F80809CB
:101DF000C2F8080BF2D20B686B676362EB6E1022BD
:101E00001A611E6916F01006FBD1122000F0AAFE1E
:101E1000D4F8003823F4FE63C4F80038A36943F40F
:101E2000402343F01003A3610923C4F81038C4F819
:101E30001438094BEB60094BC4F8106BC4F8003B35
:101E4000C4F81069C4F800396B6F03F1100243F451
:101E500080136A67A362F8BDDC330008408000107D
:101E6000C26E90F86610D2F8003823F4FE6343EA9D
:101E70000113C2F8003870472DE9F0410EB200EBB3
:101E800086080D46D8F80C100F6807F00303022BE4
:101E900050D0032B50D03D4A3D4F012B18BF174661
:101EA000C46E4FEA451E04EB0E030022C3F8102B4C
:101EB0008A6905F1100C002A40D04A8A05F15803BE
:101EC0005B013A43E2500123D4F81C2803FA0CF3D7
:101ED0001343A6444A69C4F81C380023CEF81039CD
:101EE00005F13F03002A39D00A8A898B920801291B
:101EF00088BF4A43416F04EB8303561841EA02420C
:101F0000466729465A602046FFF7E2FDD8F80C30B4
:101F10001B8A43EA85531F4305F148035B01E750E1
:101F20000123D4F81C2803FA05F51543C4F81C58FE
:101F3000BDE8F081174FB3E7174FB1E704EB461345
:101F4000D3F8002B22F40042C3F8002BD4F81C284D
:101F5000012303FA0CF322EA0303BAE704EB830339
:101F60000E4A5A6004EB461629462046FFF7B0FD9C
:101F7000D6F8003923F40043C6F80039D4F81C38E9
:101F8000012202FA05F523EA0505CFE700800010DB
:101F9000008004100080081000800C100004000273
:101FA000026F12684267FFF775BD00005831C36EBB
:101FB00049015B5813F4004004D013F4001F14BF10
:101FC00001200220704700004831C36E49015B5870
:101FD00013F4004004D013F4001F14BF01200220AA
:101FE0007047000000EB8101CB68196A0B68136031
:101FF0004B6853607047000000EB810330B5DD682B
:10200000AA691368D36019B9402B84BF40231360B9
:102010006B8A1468C26E1C44013CB4FBF3F4634346
:10202000033323F0030302EB411043EAC44343F0BC
:10203000C043C0F8103B2B6803F00303012B09B227
:102040000ED1D2F8083802EB411013F4807FD0F89B
:10205000003B14BF43F0805343F00053C0F8003BF3
:1020600002EB4112D2F8003B43F00443C2F8003BBC
:1020700030BD00002DE9F041264DEE6E06EB401319
:102080000446D3F8087BC3F8087B38070AD5D6F88E
:102090001438190706D505EB84032146DB6828466A
:1020A0005B689847FA0732D5D6F81438DB072ED587
:1020B00014B995F84C3053B305EB8403D968C4B90F
:1020C0008B69488A5E68B6FBF0F200FB126282B947
:1020D0001868DA6890420CD2121A83E81400FFF7ED
:1020E000D3FC21460B48FFF787FF84F31188BDE836
:1020F000F081012303FA04F26B8923EA02036B8166
:10210000CB6823B121460348BDE8F0411847BDE83C
:10211000F08100BF100E012000EB810370B5DD6877
:10212000C36E6C692668E6604A0156BB1A444FF4D8
:102130000020C2F810092A6802F00302012A0AB23C
:102140000ED1D3F8080803EB421410F4807FD4F8C2
:10215000000914BF40F0805040F00050C4F800095E
:1021600003EB4212D2F8000940F00440C2F8000923
:10217000D3F83408012202FA01F10143C3F83418FC
:1021800070BD19B9402E84BF4020206020682E8A7F
:10219000841940F00050013C1A44B4FBF6F440EAC4
:1021A000C440C6E72DE9F041274CE66E06EB40132C
:1021B0000546D3F80879C3F80879F90719D5D6F890
:1021C0001038DA0715D504EB8003D9684B69186815
:1021D000DA6890422AD2121A4FF000081A60C3F847
:1021E0000480FFF751FC29462046FFF795FF88F34E
:1021F00011883B0618D5D6F83428012303FA05F5D3
:10220000154211D0FFF740FCA36F10482B43A36782
:10221000D6F8343823EA0505C6F834580021FEF70D
:10222000B1FF002383F31188BDE8F081012303FA95
:1022300005F2238923EA020323818B68002BD8D07F
:10224000294620469847D4E7100E01208C0E012025
:102250002DE9F74F8948C46E6669A3691E4016F4DC
:10226000805F6661054608D000238367FFF7E6F9C3
:1022700003B0BDE8F04F00F0C9BC002E12DAD4F86C
:10228000003E7E4899071EBFD4F8003E23F00303AA
:10229000C4F8003ED4F8043843F00103C4F804380D
:1022A000FFF7F8F9320504D500237448AB67FFF750
:1022B000E5F9B3040CD5D4F8083813F0060FE36839
:1022C00023F470530CBF43F4105343F4A053E36062
:1022D000370704D56B68DB680BB168489847F00294
:1022E00061D4B1020CD5D5F86C80DFF890A100273D
:1022F0004FF001092B6F9B68F9B28B4280F0A180EF
:10230000F2060CD5FFF7C0FBA3695D4823F010036C
:10231000A3610021FEF736FF002383F31188330306
:10232000D4F818481DD5E70302D50020FFF7A2FE18
:10233000A50302D50120FFF79DFE600302D5022010
:10234000FFF798FE210302D50320FFF793FEE20278
:1023500002D50420FFF78EFEA30202D50520FFF769
:1023600089FE770384D5E60702D50020FFF71AFF20
:10237000A50702D50120FFF715FF600702D502204F
:10238000FFF710FF210702D50320FFF70BFFE2063E
:1023900002D50420FFF706FFA3067FF569AF0520ED
:1023A000FFF700FF64E7D5F86C90DFF8D4A04FF09A
:1023B00000082A6F92685FFA88F39A4291D309EB7A
:1023C0004312D2F8001901F44021B1F5802F35D124
:1023D000D2F80019002931DAD2F8001941F0904101
:1023E000C2F80019D2F800190029FBDB1946E86E83
:1023F0000193FFF76DFB019B012202FA03FB2A897F
:102400006FEA0B073A402A8105EB8302D268926893
:1024100012B1194619489047FFF736FBD9F83438FE
:102420001F40AB6FC9F8347843EA0B0300215046D4
:10243000AB67FEF7A7FE002383F3118808F10108BC
:10244000B7E708EB4112D2F8003B03F44023B3F5A1
:10245000802F10D1D2F8003B002B0CDA6A8909FAE0
:1024600001F322EA03036B8105EB8103DB68DB6880
:102470000BB15046984701373CE700BF100E0120D2
:102480008C0E0120C36E03EB4111D1F8003B43F4E5
:102490000013C1F8003B7047C36E03EB4111D1F844
:1024A000003943F40013C1F800397047C36E03EBE1
:1024B0004111D1F8003B23F40013C1F8003B7047F1
:1024C000C36E03EB4111D1F8003923F40013C1F8B6
:1024D000003970474FF0804310B51A6992070AD54A
:1024E00000241C6172B6202383F3118862B600F0C9
:1024F000FDFA84F31188BDE8104000F087BB0000AE
:102500000E4A136C43F0010313640D4A936843F0C1
:10251000010393604FF080436B229A624FF0FF32C9
:10252000DA6200229A615A63DA605A6001225A61C3
:1025300008211A601C2000F09FBD00BF0038024037
:10254000002004E000207047FEE700007047000014
:102550004FF0FF307047000000F0CEBD08B500F02E
:1025600085FB00F07DFABDE8084000F001B90000ED
:102570007047000072B6202383F3118862B670475B
:10258000022906D0032906D00129064818BF0020D9
:10259000704705487047032A9ABF044800EBC20001
:1025A0000020704740360008F4350008300801204C
:1025B00070B5044608460D46FEF718FBC6B2204625
:1025C000013403780BB9184670BD32462946FEF730
:1025D000F5FA0028F3D1012070BD00002DE9F04F7D
:1025E00081469BB008460D461646FEF7FFFA3D4968
:1025F000C4B22846FFF7DCFF08B10434E4B23A491C
:102600002846FFF7D5FF08B11034E4B2632C01AFC0
:102610000CD8DFF8E0A0DFF8E0B03C4695F8008089
:10262000B8F1000F1CD184F8008003E02946384639
:1026300000F046FE3846FEF7D9FAC0B2431C5B00F4
:1026400089E848003370032373700023023619466B
:10265000DAB2904206F102063DD81BB0BDE8F08F19
:10266000B8F1250F32D107221E492846FEF7A6FAF7
:1026700070B9DBF800202260DBF804206260BBF850
:10268000082022819BF80A20A27207350B34C5E787
:10269000082215492846FEF791FAB8B91348A21C3A
:1026A00010F8011F124B4FEA111E01F00F011EF826
:1026B0000AE011F80A1002F802EC984202F8011C34
:1026C00002F10202ECD118340835A7E784F8008043
:1026D00001350134A2E7FA5C06F8022C06F8011C69
:1026E0000133B5E79C350008A43500081FF4F01F3E
:1026F0002BF4F01FB9350008AD35000808B5FFF719
:1027000039FF0348FEF790FE002383F3118808BDCC
:102710001811012010B50446052915D8DFE801F08D
:1027200015140315151BFFF725FF0E4A0121FEF7AF
:1027300037FF20460C4A0221FEF732FF0B48FEF716
:1027400039FE002383F3118810BDFFF713FF0748FC
:10275000FEF70CFEF5E7FFF70DFF0448FEF71EFE3F
:10276000EFE700BF4C350008703500081811012054
:1027700038B50C4D0C4C0D492A4604F10800FFF702
:102780002DFF05F1CA0204F110000949FFF726FFE9
:1027900005F5CA7204F118000649BDE83840FFF794
:1027A0001DBF00BFD815012030080120CC3500081E
:1027B000D6350008A4350008BFF34F8F024AD3680E
:1027C000DB03FCD4704700BF003C024008B5074B58
:1027D0001B7853B9FFF7F0FF054B1A69002ABFBFFA
:1027E000044A5A6002F188325A6008BD3618012046
:1027F000003C02402301674508B5054B1B7833B9FF
:10280000FFF7DAFF034A136943F00043136108BD81
:1028100036180120003C0240072870B513D80B4A37
:102820000B4C137863B90B4E4FF0006144F8231042
:1028300056F823500133082B2944F7D10123137094
:1028400054F8200070BD002070BD00BF5818012052
:102850003818012060360008014B53F820007047FB
:102860006036000808207047072810B5044601D9D3
:10287000002010BDFFF7D0FF064B53F8243018445A
:10288000C21A0BB9012010BD12680132F0D1043B0D
:10289000F6E700BF60360008072810B504462FD8B9
:1028A000FFF78AFFFFF792FF1649F323CB60FFF78C
:1028B00083FFC300DBB243F4007343F002030B61F8
:1028C0000B6943F480330B61FFF776FFFFF7A4FF3A
:1028D0000D4B53F824300344BFF34F8F0B4A9842FB
:1028E0000AD3BFF34F8FBFF36F8FFFF785FF2046EB
:1028F000BDE81040FFF7B8BFC2F85C022030EEE739
:10290000002010BD003C02406036000800ED00E0F1
:102910002DE9F047D40715464DD41318B3F1016FD4
:1029200049D2324B1B68DA0745D5314CFFF74EFFD1
:10293000F323E360FFF740FF2F46401A40F20129DE
:10294000032F884601EB000618D8294C40F20119E4
:102950007B1A4344012B01EB000623692FD823F097
:1029600001032361FFF748FF2846BDE8F08736687A
:1029700051F8043CB34218D1043FE1E7B307E4D176
:10298000236923F440732361236943EA0903236124
:102990000431D8F800303360BFF34F8FFFF70CFFDE
:1029A000E368002BE3D0F323E360236923F0010302
:1029B0002361FFF721FF4FF0FF30BDE8F08723F4DC
:1029C00040732361236943EA090323618A4631F88E
:1029D000023B3380BFF34F8FFFF7EEFE3688BAF825
:1029E0000030B6B2B342B3D0DFE700BF00380240D8
:1029F000003C0240084908B50B7828B153B9FFF7ED
:102A0000E5FE01230B7008BD23B1BDE80840087046
:102A1000FFF7F2BE08BD00BF36180120014B186D4C
:102A2000704700BF00280040094B1A6F120407D4FA
:102A30001A6F42F400721A671A6F42F400421A6762
:102A4000044A136843F480731360034B186570479E
:102A5000003802400070004000280040FEE70000FF
:102A600010B51A4CFEF768FAFEF7E2F900F0ACF880
:102A7000802217492046FEF71FFB012344F8180C5B
:102A80000374144B144AD96821F4E0610904090C59
:102A90000A431249DA60CA6842F08072CA60104A7A
:102AA0001049C2F8B01F116841F0010111601022F5
:102AB000DA77202283F82220002383F3118862B67C
:102AC0000948BDE81040FEF725BB00BFF00D01200E
:102AD0008036000800ED00E00003FA05F0ED00E0AC
:102AE000001000E055CEACC5883600082DE9F8434B
:102AF0001B4C4FF0804300256769586A04F11408A5
:102B00002E46226ABB68811A8B420CD96169414505
:102B100024D013441B1A022B2CBFC0180230BDE86E
:102B2000F843FEF70DBD134423623B68D7F80C90C1
:102B3000C3F8048043456361FD6001D1FEF7FAFCF0
:102B400086F311883869C84772B6202383F3118849
:102B500062B64FF080436769586AD2E7BDE8F883F0
:102B6000C80D0120034B59685A68521A9042FBD88D
:102B7000704700BF001000E083691943037C816146
:102B80000A2B03D14369194205D170470B2B06D19B
:102B900043698B4303D100234361FEF7D5B97047E6
:102BA00070B5046805460E46AC4200D170BDE368BE
:102BB0003343E36016B12269134203D0A168606811
:102BC000FFF7DAFF2468EFE7034B044A1A60044B6F
:102BD000044A1A60704700BF5C1A0120601A012085
:102BE000581A01200000052080B5074A536823F0D9
:102BF000010300AF5360EFF30983683383F309885F
:102C0000002383F3118880BD30EF00E098B500AF5A
:102C100072B6202383F3118862B6104B5B6813F4FD
:102C2000006318D0F1EE103AEFF309844FF080738F
:102C300044F84C3C0A4BDB6844F8083CA4F16803B8
:102C400083F30988FEF708FA18B1064B44F8503CA4
:102C500098BD054BFAE783F3118898BD00ED00E0BD
:102C600030EF00E0410300084403000808B500F01D
:102C700019FA064800F0C8FAFEF76CFCFEF72EFBC6
:102C8000FFF776FCBDE80840FEF74ABC18340008A0
:102C900072B6202383F3118862B6704730B5039C67
:102CA0000172043304FB0325C361049B0363002109
:102CB000059B00604060C160426102618561046201
:102CC00042628162C162436330BD00000022416AFA
:102CD00041610161C2608262C2626FF00101FEF770
:102CE00077BA000003694269934203D1C2680AB10E
:102CF00000207047181D704703691960C2680132CF
:102D0000C260C269134482690361934224BF436A6B
:102D100003610021FEF750BA38B504460D46E3685A
:102D20003BB16269131D1268A3621344E362002081
:102D300038BD237A33B929462046FEF72DFA0028FC
:102D4000EDDA38BD6FF00100FBE70000C368C2692F
:102D5000013BC3604369134482694361934224BFCA
:102D6000436A436100238362036B03B118477047D2
:102D700070B50446FFF78CFF866A3EB9FFF7CCFFBB
:102D8000054618B186F31188284670BDA36AE26A29
:102D900013F8015BA362934202D32046FFF7D6FFEC
:102DA000002383F31188EFE72DE9F74F4FF08048B8
:102DB0001F4604460E469146FFF76AFFD8F82430B6
:102DC0000025FB18009307F1FF3AAB46A36AABB9A5
:102DD0001AF1030F06D939462046FFF79DFF68B167
:102DE000002305E0D8F82410009A511A8F42F3D23C
:102DF00083F31188284603B0BDE8F08FA16AE36A27
:102E0000A9EB05025B1A934228BF1346402B1BD93E
:102E1000334601F1400251F8040B43F8040B914290
:102E2000F9D1A36A40334036A3624035A26AE36A0F
:102E30009A4202D32046FFF789FF8BF311884D4554
:102E4000D8D2FFF725FFC1E71A4630460193FDF7B8
:102E5000ABFE019BA26A1A441E44A2621D44E5E730
:102E600010B5029C0172043303FB0421C3610023EB
:102E70008362C362039B0363049B00604060C46081
:102E800042610261816104624262436310BD0000DD
:102E9000026AC260426A4261026100228262C262C8
:102EA0006FF00101FEF794B9436902699A4203D1B8
:102EB000C2680AB100207047184650F8043B0B6006
:102EC00070470000C368C2690133C360436913449B
:102ED00082694361934224BF436A43610021FEF744
:102EE0006BB9000038B504460D46E3683BB1236971
:102EF0001A1DA262E2691344E362002038BD237AFE
:102F000033B929462046FEF747F90028EDDA38BDE7
:102F10006FF00100FBE7000003691960C268013A25
:102F2000C260C269134482690361934224BF436A49
:102F3000036100238362036B03B1184770470000ED
:102F400070B504460E46FFF7A3FE856A35B91146F3
:102F5000FFF7C8FF10B185F3118870BDA36A1E701A
:102F6000A36AE26A01339342A36204D3E169204673
:102F70000439FFF7D1FF002080F3118870BD0000F5
:102F80002DE9F74F4FF080481F4604460D46914605
:102F9000FFF77EFED8F824300026FB18009307F1D7
:102FA000FF3AB346A36AABB91AF1030F06D9394603
:102FB0002046FFF797FF68B1002305E0D8F82410FA
:102FC000009A511A8F42F3D283F31188304603B02E
:102FD000BDE8F08FA06AE36AA9EB06021B1A9342D0
:102FE00028BF1346402B1BD905F1400355F8042B8D
:102FF00040F8042B9D42F9D1A36A4033A3624036C6
:10300000A26AE36A9A4204D3E16920460439FFF7D1
:1030100083FF8BF311884E45D8D2FFF739FEC1E705
:103020001A4629460193FDF7BFFD019BA26A1A4487
:103030001D44A2621E44E3E7026943699A4203D138
:10304000C3681BB9184670470023FBE7836A002B4F
:10305000F8D0043B9B1AF5D01360C368013BC360F2
:10306000C3691A44836902619A4224BF436A0361B7
:10307000002383620123E5E700F1604300F01F02B3
:10308000400903F5614309018000C9B200F16040C5
:1030900083F8001300F5614001239340C0F88031AC
:1030A00003607047124B00211A694FF0FF321A611A
:1030B000196158695A615961186A60F08050186244
:1030C0001962586A5A620B4A5962106840F480705B
:1030D0001060186F00F44070B0F5007F1EBF4FF411
:1030E000803018671967536823F400735360704782
:1030F0000038024000700040364B4FF080521A6496
:10310000354A4FF4404111601A6842F001021A60DA
:103110001A689207FCD59A6822F003029A609A68AE
:103120009A602C4B19469A6812F00C02FBD1186871
:1031300000F0F90018609A601A6842F480321A6050
:103140000B689B03FCD54B6F43F001034B67214B8E
:103150005A6F9007FCD5214A5A601A6842F0807273
:103160001A601D4B1A4659684904FCD5196841F488
:10317000803119605368D803FCD5136843F40033D9
:103180001360154A53689903FCD5124B1A689201D3
:10319000FCD5134A9A6040F20112C3F88C20002239
:1031A000C3F890200F4A40F2093111609A6842F04A
:1031B00002029A60074B9A6802F00C02082AFAD1C0
:1031C0005A6C42F480425A645A6E42F480425A6603
:1031D000704700BF0038024000700040086C400992
:1031E00000948838003C02404B6843608B688360E1
:1031F000CB68C3600B6943614B6903628B694362AF
:103200000B68036070470000214B0246186B10B535
:1032100040F2FF7420431863196D1E48214319655D
:103220001146FFF7E1FF1C4802F11C01FFF7DCFF2C
:103230001A4802F13801FFF7D7FF194802F154018B
:10324000FFF7D2FF174802F17001FFF7CDFF1648D4
:1032500002F18C01FFF7C8FF144802F1A801FFF743
:10326000C3FF134802F1C401FFF7BEFF114802F18A
:10327000E001FFF7B9FF104802F1FC01FFF7B4FFCE
:103280000E4802F58C71BDE81040FFF7ADBF00BFDE
:1032900000380240000002400004024000080240E2
:1032A000000C0240001002400014024000180240CE
:1032B000001C02400020024000240240002802407E
:1032C00080EA0102844612F0030F4FD111F0030F80
:1032D00032D14DF8044D11F0040F51F8043B0BD0DE
:1032E000A3F101329A4312F0803F04BF4CF8043B33
:1032F00051F8043B16D100BF51F8044BA3F1013241
:103300009A4312F0803FA4F101320BD14CF8043BF8
:10331000A24312F0803F04BF51F8043B4CF8044B29
:10332000EAD023460CF8013B13F0FF0F4FEA33239A
:10333000F8D15DF8044B704711F0010F06D011F879
:10334000012B0CF8012B002A08BF704711F0020F67
:10335000BFD031F8022B12F0FF0F16BF2CF8022B52
:103360008CF8002012F47F4FB3D1704711F8012B75
:103370000CF8012B002AF9D1704700BF121012136C
:103380001211000053544D3332463F3F3F3F3F3F01
:103390000053544D333246375B347C355D780053EF
:1033A000544D333246375B367C375D780000000081
:1033B0005912000845120008811200086D12000819
:1033C0007912000865120008511200083D12000829
:1033D00000000000010000000000000000000000EC
:1033E000A916000881190008191A000840004000B9
:1033F0000011012000110120010000001011012026
:103400008000000040010000050000007573625F4D
:1034100070756D70000000001000802A0000000030
:10342000AAAAAAAA00000000FFFF000000000000F6
:1034300000A00A000000000000000000AAAAAAAA3A
:1034400000000000FFFF000000000000000000007E
:103450000000000000000000AAAAAAAA00000000C4
:10346000FFFF00000000000000000000000000005E
:1034700000000000AAAAAAAA00000000FFFF0000A6
:10348000000000000000000000000000000000003C
:10349000AAAAAAAA00000000FFFF00000000000086
:1034A000000000000000000000000000AAAAAAAA74
:1034B00000000000FFFF000000000000000000000E
:1034C0000000000000000000AAAAAAAA0000000054
:1034D000FFFF0000000000000000000000000000EE
:1034E000000000000A0000000000000003000000CF
:1034F00000000000000000000000000000000000CC
:1035000000000000000000000000000000000000BB
:1035100000000000000000000000000000000000AB
:10352000000000000000000000000000000000009B
:10353000000000000000000000000000000000008B
:103540000000000000000000000000000200000079
:103550000000000075140008DD1400084000400061
:10356000A8150120B815012002000000000000008D
:1035700003000000000000001D150008000000000E
:1035800010000000C815012000000000010000002C
:1035900000000000100E01200101020025424F41F1
:1035A000524425002553455249414C25004F4D4E6C
:1035B000494255534637563200303132333435366E
:1035C0003738394142434445460000004172647532
:1035D00050696C6F740025424F415244252D424C76
:1035E000000000001527000881250008E1130008ED
:1035F000FD26000843000000FC35000809024300D6
:10360000020100C032090400000102020100052489
:103610000010010524010001042402020524060013
:1036200001070582030800FF09040100020A0000E7
:10363000000705010240000007058102400000006C
:10364000120000004836000812011001020000407C
:10365000830440570002010203010000040309042F
:10366000008000000080000000800000008000005A
:10367000000002000000040000000400000004003C
:103680006D61696E00000000A0360008601801201E
:10369000581A0120010000005D2A00080000000007
:1036A00069646C6500000000FF000000000000007D
:1036B000843300083F0000004904000091330008F3
:1036C0003F000000510400009F3300083F0000004D
:1036D0000096000000000800040000005C360008AE
:1036E00000000000000000000000000000000000DA
:0836F0000000000000000000D2
:00000001FF
